:020000020000FC
:0200000003C03B
:1000060039C03FE53DBF34E03EBF3FEF37BB34BBB1
:1000160031EC3FBD31E03EBD30E83ABD3AE035BD9A
:100026003EE633BD30E839BFC0E6D0E0839510EF39
:100036007894C59A8823F1F3A0E6B0E0882734E0E7
:100046006AE050FF07C04FEF4D933A95E1F76A9586
:1000560049F034E040E04D933A95E1F76A9511F0A6
:1000660034E0F1CF73957E3129F7539551FD55272D
:100076007727E0CFC0E6D0E02FB608E2502E08B3CF
:100086000E7F302E0160402E38BA0991000048BA22
:1000960005BB38BA029505BB48BA5A94A9F738BACF
:1000A6001395C29A00000000C298C398103F09F049
:0C00B60002C0C39A11272FBE8395189535
:00000001FF
